:1000000092C0AAC0A9C0A8C0A7C0A7C0A5C0A4C0CC
:10001000A3C0A2C0A1C0A0C09FC09EC09DC09CC0E4
:100020009BC09AC099C000000000010101020203B8
:100030000405050607090A0B0C0E0F1112141517FB
:10004000191B1D1F212325282A2C2F313436393B1B
:100050003E414346494C4F5255585A5D6164676A68
:100060006D707376797C7F8386898C8F9295989B4F
:100070009EA2A5A7AAADB0B3B6B9BCBEC1C4C6C93D
:10008000CBCED0D3D5D7DADCDEE0E2E4E6E8EAEBAB
:10009000EDEEF0F1F3F4F5F6F8F9FAFAFBFCFDFDFC
:1000A000FEFEFEFFFFFFFFFFFFFFFEFEFEFDFDFC6D
:1000B000FBFAFAF9F8F6F5F4F3F1F0EEEDEBEAE815
:1000C000E6E4E2E0DEDCDAD7D5D3D0CECBC9C6C4D5
:1000D000C1BEBCB9B6B3B0ADAAA7A5A29E9B989568
:1000E000928F8C898683807C797673706D6A676461
:1000F000615D5A5855524F4C494643413E3B393653
:1001000034312F2C2A282523211F1D1B19171514C4
:1001100012110F0E0C0B0A09070605050403020253
:1001200001010100000011241FBECFEDCDBF10E082
:10013000A0E6B0E0EAEEF2E003C0C89531960D9279
:10014000AA37B107D1F710E0AAE7B0E001C01D92CD
:10015000A93AB107E1F76CC053CF1F920F920FB6C7
:100160000F9211242F933F934F935F936F938F932D
:100170009F93AF93BF93EF93FF9380917A00815049
:1001800080937A00882329F480917B008F5F80938D
:100190007B0010929B0010929A001092970060E0F2
:1001A00040E050E0262F3327F32FE22FE456FF4F95
:1001B00080818823D9F0F32FE22FE20FF31FAE2FB7
:1001C000BF2FA458BF4FE05AFF4F8D919C911197BC
:1001D00020813181820F931F8D939C93E92FFF27FC
:1001E000EA5DFF4FC895802D480F511D862F8F5F08
:1001F000682F8D30B8F250939B0040939A00809303
:100200009700569547955695479548BD88B58ABD40
:10021000FF91EF91BF91AF919F918F916F915F91FE
:100220004F913F912F910F900FBE0F901F901895F7
:10023000CFEDD0E0DEBFCDBF87EF88BB88E187BBC5
:100240008FE782BB11BA81EB8FBD81E08EBD80E864
:1002500089BF789480917B008823E1F3815080935B
:100260007B0086B3282F33272770307086B39927F9
:10027000807E90709595879595958795282B392B3D
:1002800080B399278F77907046E0880F991F4A9521
:10029000E1F7282B392B2095309530939900209346
:1002A000980010929600A1E0B0E0732F622F40E01A
:1002B000242F33278A2F9B2F022E02C0880F991FCD
:1002C0000A94E2F786239723F32FE22FE456FF4F99
:1002D000892B11F0A08301C01082842F8F5F482FDB
:0A02E0008D3030F380939600B5CF07
:1002EA008A080C099509270AC20A660B130CCB0C5B
:0A02FA008E0D5C0E370F1E1014115C
:00000001FF
